:020000040800F2
:1000000000060020B5050008291A0008DD190008BF
:10001000051A0008DD190008FD190008B7050008D9
:10002000B7050008B7050008B7050008A94600088D
:10003000B7050008B7050008B7050008B7050008B0
:10004000B7050008B7050008B7050008B7050008A0
:10005000B7050008B70500082D5D0008595D0008C8
:10006000855D0008B15D0008DD5D0008B70500088A
:10007000B7050008B7050008B7050008B705000870
:10008000B7050008B7050008B7050008B705000860
:10009000B7050008B7050008B7050008095E0008A5
:1000A000B7050008B7050008B7050008B705000840
:1000B000B7050008B7050008B7050008B705000830
:1000C000B7050008B7050008B7050008B705000820
:1000D000B7050008F55E0008B7050008B705000879
:1000E0006D5E0008B7050008B7050008B7050008F1
:1000F000B7050008B7050008B7050008B7050008F0
:10010000B7050008B7050008095F0008B705000833
:10011000B7050008B7050008B7050008B7050008CF
:10012000B7050008B7050008B7050008B7050008BF
:10013000B7050008B7050008B7050008B7050008AF
:10014000B7050008B7050008B7050008B70500089F
:10015000B7050008B7050008B7050008B70500088F
:10016000B7050008B7050008B7050008B70500087F
:10017000B7050008C9530008B7050008B70500080F
:10018000B7050008B7050008B7050008B70500085F
:10019000B7050008B7050008B7050008B70500084F
:1001A000B7050008B7050008B7050008B70500083F
:1001B000E15E0008B7050008B7050008B7050008AC
:1001C000B7050008B7050008B7050008B70500081F
:1001D000B7050008B5530008B7050008B7050008C3
:1001E000B7050008B7050008B7050008B7050008FF
:1001F000B7050008B7050008B7050008B7050008EF
:10020000B7050008B7050008B7050008B7050008DE
:10021000B7050008B7050008B7050008B7050008CE
:10022000B7050008B705000839480008B7050008F9
:10023000B7050008B7050008B7050008B7050008AE
:10024000B7050008B7050008B7050008B70500089E
:10025000B7050008B7050008B7050008B70500088E
:10026000B7050008B7050008B7050008B70500087E
:10027000B7050008B7050008B7050008B70500086E
:10028000B7050008B7050008B7050008B70500085E
:10029000B7050008B7050008B7050008B70500084E
:1002A0009D070008B519000895240008000000000B
:1002B00053B94AB9002908BF00281CBF4FF0FF31CD
:1002C0004FF0FF3000F074B9ADF1080C6DE904CEC9
:1002D00000F006F8DDF804E0DDE9022304B0704721
:1002E0002DE9F047089D04468E46002B4DD18A42E9
:1002F000944669D9B2FA82F252B101FA02F3C2F11C
:10030000200120FA01F10CFA02FC41EA030E9440AC
:100310004FEA1C48210CBEFBF8F61FFA8CF708FBCD
:1003200016E341EA034306FB07F199420AD91CEBA5
:10033000030306F1FF3080F01F81994240F21C81D7
:10034000023E63445B1AA4B2B3FBF8F008FB10331F
:1003500044EA034400FB07F7A7420AD91CEB040454
:1003600000F1FF3380F00A81A74240F20781644424
:10037000023840EA0640E41B00261DB1D4400023A9
:10038000C5E900433146BDE8F0878B4209D9002D0D
:1003900000F0EF800026C5E9000130463146BDE897
:1003A000F087B3FA83F6002E4AD18B4202D3824201
:1003B00000F2F980841A61EB030301209E46002DB0
:1003C000E0D0C5E9004EDDE702B9FFDEB2FA82F205
:1003D000002A40F09280A1EB0C014FEA1C471FFA63
:1003E0008CFE0126200CB1FBF7F307FB131140EA4A
:1003F00001410EFB03F0884208D91CEB010103F117
:10040000FF3802D2884200F2CB804346091AA4B2D8
:10041000B1FBF7F007FB101144EA01440EFB00FEAC
:10042000A64508D91CEB040400F1FF3102D2A64511
:1004300000F2BB800846A4EB0E0440EA03409CE7B0
:10044000C6F12007B34022FA07FC4CEA030C20FA5D
:1004500007F401FA06F31C43F9404FEA1C4900FA7D
:1004600006F3B1FBF9F8200C1FFA8CFE09FB1811FA
:1004700040EA014108FB0EF0884202FA06F20BD96D
:100480001CEB010108F1FF3A80F08880884240F2BD
:100490008580A8F102086144091AA4B2B1FBF9F001
:1004A00009FB101144EA014100FB0EFE8E4508D9FC
:1004B0001CEB010100F1FF346CD28E456AD9023881
:1004C000614440EA0840A0FB0294A1EB0E01A14266
:1004D000C846A64656D353D05DB1B3EB080261EBD4
:1004E0000E0101FA07F722FA06F3F1401F43C5E9AE
:1004F000007100263146BDE8F087C2F12003D840E4
:100500000CFA02FC21FA03F3914001434FEA1C4725
:100510001FFA8CFEB3FBF7F007FB10360B0C43EA17
:10052000064300FB0EF69E4204FA02F408D91CEBC7
:10053000030300F1FF382FD29E422DD902386344C5
:100540009B1B89B2B3FBF7F607FB163341EA034165
:1005500006FB0EF38B4208D91CEB010106F1FF38B4
:1005600016D28B4214D9023E6144C91A46EA0046AB
:1005700038E72E46284605E70646E3E61846F8E63D
:100580004B45A9D2B9EB020864EB0C0E0138A3E786
:100590004646EAE7204694E74046D1E7D0467BE767
:1005A000023B614432E7304609E76444023842E7DF
:1005B000704700BF02E000F000F8FEE772B63A486C
:1005C00080F30888394880F3098839484EF6085185
:1005D000CEF20001086040F20000CCF200004EF6BE
:1005E0003471CEF200010860BFF34F8FBFF36F8FFD
:1005F00040F20000C0F2F0004EF68851CEF2000149
:100600000860BFF34F8FBFF36F8F4FF00000E1EE34
:10061000100A4EF63C71CEF200010860062080F30D
:100620001488BFF36F8F04F0FDF804F09FF805F015
:100630003BF94FF055301F491B4A91423CBF41F8EE
:10064000040BFAE71C49194A91423CBF41F8040BDC
:10065000FAE71A491A4A1B4B9A423EBF51F8040B5B
:1006600042F8040BF8E700201749184A91423CBFB2
:1006700041F8040BFAE704F0B7F805F08BF9144CD5
:10068000144DAC4203DA54F8041B8847F9E700F034
:100690004FF8114C114DAC4203DA54F8041B884753
:1006A000F9E704F09FB800000006002000220020B7
:1006B0000000000800000020000600202867000855
:1006C00000220020C8220020C8220020D849002093
:1006D000A0020008AC020008AC020008AC0200084E
:1006E0002DE9F04F2DED108AC1F80CD0D0F80CD0C8
:1006F000BDEC108ABDE8F08F002383F311882846F3
:10070000A047002003F008FAFEE703F037F900DF06
:10071000FEE70000054B10B504460360806810B189
:1007200003685B689847204610BD00BF0863000857
:1007300038B503F0DFFE054603F0ACFF0446F0B920
:10074000144B9D421DD001339D4241F2883512BFAA
:10075000044600250124002003F0D6FE0CB100F071
:100760009FF80D4C00F018FF00F0C2FD204601F08C
:10077000C9FC40B944F6206003F0D4F9F6E700253F
:10078000E9E70546E7E7284600F046F900F088F873
:10079000F9E700BF010007B0C82200200448054B5C
:1007A000054A036000230549836005F007BC00BFCC
:1007B000C822002008630008D8240020150700087C
:1007C00008B500F061FDA0F120035842584108BD72
:1007D00007B5042101900DEB010000F073FD03B09B
:1007E0005DF804FB07B541F21203022101A8ADF840
:1007F000043000F067FD03B05DF804FB38B520233A
:1008000083F311881748C3680BB103F023FA002360
:10081000154A4FF47A71134803F0E0F9002383F38B
:100820001188124C236813B12368013B236063686D
:1008300013B16368013B63600D4D2B7833B9636876
:100840007BB9022000F012FE322363602B78032B69
:1008500007D163682BB9022000F008FE4FF47A73C9
:10086000636038BD58230020FD0700087424002071
:100870006C230020084B187003280CD8DFE800F028
:1008800008050208022000F0E9BD022000F0DCBDEE
:10089000024B00225A6070476C2300207424002011
:1008A000F7B5564801A901F0A5FD002800F0A38086
:1008B000534B544A1C461968013100F099800433A7
:1008C0009342F8D16268504B9A4240F291804F4B6C
:1008D000DB6803F1104303F580139A4280F08880AF
:1008E000002000F01FFD0220FFF7C4FF484B00214D
:1008F000D3F8E820C3F8E810D3F81021C3F810119A
:10090000D3F81021D3F8EC20C3F8EC10D3F814215D
:10091000C3F81411D3F81421D3F8F020C3F8F01061
:10092000D3F81821C3F81811D3F81821D3F8802070
:1009300042F00062C3F88020D3F8802022F00062E9
:10094000C3F88020D3F88020D3F8802042F00072D2
:10095000C3F88020D3F8802022F00072C3F88020F2
:10096000D3F8803072B64FF0E023C3F8084DD4E9D5
:100970000004BFF34F8FBFF36F8F264AC2F8841075
:10098000BFF34F8F536923F480335361BFF34F8F0D
:10099000D2F8803043F6E076C3F3C905C3F34E3393
:1009A0005B0103EA060C29464CEA81770139C2F85B
:1009B0007472F9D2203B13F1200FF2D1BFF34F8FA5
:1009C000BFF36F8FBFF34F8FBFF36F8F536923F464
:1009D000003353610023C2F85032BFF34F8FBFF38F
:1009E0006F8F202383F31188854680F30888204782
:1009F000024801F05FF803B0F0BD00BFC82200203C
:100A00000000109020001090FFFF0F9000220020A7
:100A10000044025800ED00E02DE9F04FB34B9FB0C9
:100A20002022FF21089016A89E68DB68079300F03B
:100A30005DFDAF4A1378A3B90121AE481170C360C0
:100A4000202383F31188C3680BB103F003F900235B
:100A5000A94A4FF47A71A74803F0C0F8002383F342
:100A60001188089B13B1A54B089A1A60A44A137801
:100A7000032B03D000231370A04A53600023089D6A
:100A8000A04F98469B46CDE90533012000F0E6FCD7
:100A900025B19A4B1B68002B00F08783002000F0E3
:100AA000F3FB0E900E9B002BF2DB012000F0CCFC40
:100AB0000E9B213B1F2BE8D801A252F823F000BF68
:100AC000410B0008690B0008030C00088B0A0008A2
:100AD0008B0A00088B0A0008EF0E0008ED100008D2
:100AE000850F00086B10000891100008B71000086F
:100AF0008B0A0008C91000088B0A0008351100088D
:100B0000E10B00088B0A0008B1110008A10C0008D5
:100B1000D90D00088B0A0008E10F00088B0A0008B5
:100B20008B0A00088B0A00088B0A00088B0A000851
:100B30008B0A00088B0A00088B0A0008030C0008C7
:100B40000220FFF73DFE002840F05B83089B022156
:100B5000069A11A8002A08BF1D4641F21233ADF8CB
:100B6000443000F0AFFB90E74FF47A7000F08CFB5C
:100B7000041EEBDB0220FFF723FE0028E6D0013C39
:100B8000052C00F24083DFE804F0030A0D1013394E
:100B90000523042111A8119300F094FB17E0042110
:100BA0005248F9E704215848F6E704215748F3E78B
:100BB0004FF01C09484609F1040900F0B5FB042177
:100BC000119011A800F07EFBB9F12C0FF2D1012099
:100BD000059B4FF0000B00FA04F41C43E3B20593AD
:100BE00000F0D0FCB8F1000F05D0059B03F00B031B
:100BF0000B2B08BF0025FFF7F5FD46E7042144480D
:100C0000CAE7B8F1000FA1D0059B03F00B030B2B33
:100C10009CD10220FFF7D4FD0446002896D0012085
:100C20004FF0000800F07EFB0220FFF723FE5FFA82
:100C300088F9484600F086FB0546B8B10E9948464B
:100C400008F10108A1F140025142514100F08AFB34
:100C50000028ECD10546069441F21213022111A896
:100C6000A046ADF8443000F02DFB0EE72E46DFF82D
:100C70007C800120FFF7FEFDD8F80830B34207D989
:100C8000304600F051FB013040F0C0820436F3E7FB
:100C900000261B4BA04606941E70184B5E609FE713
:100CA000B8F1000F3FF452AF059B03F00B030B2B81
:100CB0007FF44CAF64210FA800F0FAFA81460028B7
:100CC0007FF444AF0220FFF77BFD044600283FF489
:100CD0003DAF3A6A7B6A0F9953438DF837908B4248
:100CE0001AD20C4800F0CCFB30E700BF00220020F5
:100CF0007024002058230020FD07000874240020E1
:100D00006C230020C822002004220020082200209A
:100D10000C220020006100084FF4801AAC48C8463D
:100D2000BAFBF2FA00F0ACFBFFF75CFD01210DF11C
:100D3000370000F0C7FA0F9B434541D9002310AAA2
:100D400051463846CDE9103311AB00F0B7FE00280C
:100D500082D000F071FE109B00EB030901210DF120
:100D6000370000F0AFFA00F067FE484520D938465A
:100D700001F0DAF880B964210F9B96480AF1010A64
:100D800001FB08F1B1FBF3F18DF83710C9B200F0A7
:100D900077FB3B6A9844CEE700F04EFE119B184467
:100DA00048453FF659AF00F047FE109B00EB0309A2
:100DB000109B4FF47A70A3FB000302F0B3FECDE763
:100DC000642301210DF13700A0468DF8373000F083
:100DD00079FA0023079303E7B8F1000F3FF4B6AEAA
:100DE000059B03F00B030B2B7FF4B0AE0220FFF743
:100DF00041FD322000F048FAB0F1000AFFF6A6AE3D
:100E0000079BD14653440993734B099ADB689A4276
:100E10003FF69CAEBAF5807F3FF798AE6F4A00244C
:100E2000A2450A920EDD4FF47A7000F02DFA0E9072
:100E30000E9B002BFFF68AAE0E9B01340A9A02F835
:100E4000013BEDE7C820FFF7BBFC044600283FF458
:100E50007DAE079B1F2B11D8C3F1200223F00300A6
:100E600016AB5E495245184428BF52460A9200F01C
:100E70000BFB0A9AFF21594800F038FB00239846E3
:100E8000CDE91033079B03F580130B93B9F1000FE5
:100E900002D1A046099B9DE711AB504A0B993846F9
:100EA000029310AB4244414401930FAB00934B4675
:100EB00001F00CFA00283FF4CFAE00F0BFFD0F9B0D
:100EC00082460A919844A9EB030900F0B7FD109BF4
:100ED0000A9A13EB0A0342F10002834272EB010308
:100EE000F3D2384601F020F80028EED1CEE7B8F171
:100EF000000F3FF42BAE059B03F00B030B2B7FF48D
:100F000025AE0220FFF7B6FC322000F0BDF9B0F1AB
:100F1000000AFFF61BAE1AF003047FF417AE2E4A48
:100F20000AEB0603926893423FF610AEBAF5807F53
:100F30003FF70CAEDFF8A490A2450DDD4FF47A70B8
:100F400000F0A2F90E900E9B002BFFF6FFAD0E9B5A
:100F5000013409F8013BEFE7C820FFF731FC0446F4
:100F600000283FF4F3ADCAF387021C4930464FEA2C
:100F7000AA0900F0C3FA804600283FF46DAE06EBE4
:100F800089062DE60220FFF71BFC00283FF4DEADAA
:100F900000F006FA00283FF4D9AD4FF00009DFF861
:100FA00038A04C46DAF808304B450CD9484609F1D0
:100FB000040900F0B9F90422119011A9204601F0AA
:100FC0008FFA0446EEE72046FFF702FC08E600BF72
:100FD000256100083D6100080022002070230020E8
:100FE000642110A800F064F9044600287FF4AEAD37
:100FF0000220FFF7E5FB00283FF4A8AD109BA146B7
:1010000003F0030A1099A1EB0A01A1421BD91F2C7E
:1010100011D8169B01330ED024F003031EAA1344EB
:1010200053F8203C11934846042211A9043401F0DE
:1010300057FA8146E6E7042311AA04F580113846E1
:1010400001F090F9EFE7BAF1000F0CD0534611AA66
:1010500001F58011384601F085F94846524611A93C
:1010600001F03EFA81464846AEE70023642111A80C
:10107000119300F01DF900287FF468AD0220FFF7FE
:101080009FFB00283FF462AD119800F07FF99BE7C9
:101090000023642111A8119300F00AF900287FF4BD
:1010A00055AD0220FFF78CFB00283FF44FAD11989F
:1010B00000F06EF988E70220FFF782FB00283FF47A
:1010C00045AD00F07DF97FE70220FFF779FB0028AE
:1010D0003FF43CAD11A9142000F078F90990FFF716
:1010E00077FB099911A800F0EDF879E5322000F0BE
:1010F000CBF8041EFFF62AADA3077FF427AD444AC0
:1011000004EB0B03926893423FF620AD0220FFF7F9
:1011100057FB00283FF41AAD24F003045C44A345B8
:101120003FF45EAD58460BF1040B00F0FDF8FFF7FD
:101130004FFBF4E74FF47A70FFF742FB00283FF4CF
:1011400005AD00F02DF980B1169B013328D011AB0D
:1011500016AA4FF480113846029310AB01930FABDF
:101160000093202301F0B2F808B9444674E500F07A
:1011700065FC284E04460D4600F060FC109B1B19D0
:1011800045F10002834272EB0103F5D2304600F0D4
:10119000CBFE0028F0D12022FF2116A800F0A6F9EE
:1011A000FFF720FB1C4802F0BDFC1FB0BDE8F08F2C
:1011B000B8F1000F3FF4CAAC059B03F00B030B2BF7
:1011C0007FF4C4AC0023642111A8119300F070F8DF
:1011D000044600287FF4BAAC0220FFF7F1FA8146FA
:1011E00000283FF4B3ACFFF7FDFA41F2883002F07B
:1011F00099FC119800F012FAC846254600F0C2F991
:1012000043E48046ECE44FF0000B9FE4069423E5B2
:1012100000220020C8220020A08601002DE9F84FFE
:101220004FF47A7306460D46002402FB03F7DFF8FD
:101230005080DFF8509098F900305FFA84FA5A1C19
:1012400001D0A34212D159F824002A46314603683E
:10125000D3F820B03B46D847854207D1074B012041
:1012600083F800A0BDE8F88F0124E4E7002CFBD050
:101270004FF4FA7002F056FC0020F3E7C02400207F
:101280001022002014220020002307B5024601216D
:101290000DF107008DF80730FFF7C0FF20B19DF872
:1012A000070003B05DF804FB4FF0FF30F9E70000E2
:1012B0000A46042108B5FFF7B1FF80F00100C0B273
:1012C000404208BD074B0A4630B41978064B53F824
:1012D0002140014623682046DD69044BAC4630BC02
:1012E000604700BFC024002014220020A086010017
:1012F00070B50A4E00240A4D02F0E2FE30802868E4
:101300003388834208D902F0D7FE2B6804440133A6
:10131000B4F5003F2B60F2D370BD00BFC2240020A3
:101320007C24002002F080BF00F1006000F5003056
:101330000068704700F10060920000F5003002F094
:10134000F7BE0000054B1A68054B1B889B1A8342A9
:1013500002D9104402F0B0BE002070477C24002067
:10136000C224002038B50446074D29B1286820441E
:10137000BDE8384002F0ACBE2868204402F0A2FE6E
:101380000028F3D038BD00BF7C2400200020704727
:1013900000F1FF5000F58F10D0F8000870470000F2
:1013A000064991F8243033B100230822086A81F8F5
:1013B0002430FFF7BFBF0120704700BF802400200A
:1013C000014B1868704700BF0010005C1B4B0246C1
:1013D000F0B518681A4BC0F30B06000C1F885C6848
:1013E000BE4293F9085003D09F89BE4203D10C330B
:1013F0005C6893F908500426124B1F880433874217
:1014000008BF13F9025C013EF7D1013A013C0B46DB
:101410000A44934207D214F9016F581C2EB10346B7
:1014200000F8016CF5E7184605E02C2482421C7098
:1014300001D9981C5D70401AF0BD00BF0010005C1F
:101440001C22002068610008022803D1024B4FF4DF
:1014500000229A61704700BF00100258022802D192
:10146000014B08229A61704700100258022804D1EB
:10147000024A536983F00803536170470010025811
:101480000FB404B070470000002310B5934203D09E
:10149000CC5CC4540133F9E710BD0000013810B52D
:1014A00010F9013F3BB191F900409C4203D11AB1C0
:1014B0000131013AF4E71AB191F90020981A10BDF0
:1014C0001046FCE70138013910F9013F11F9012FED
:1014D0000BB19342F8D0981A7047000003460246B9
:1014E000D01A12F9011B0029FAD1704702440346B1
:1014F000934202D003F8011BFAE770472DE9F84345
:101500001F4D14460746884695F8242052BBDFF845
:1015100070909CB395F824302BB92022FF214846C7
:101520002F62FFF7E3FF95F824004146C0F108025F
:1015300005EB8000A24228BF2246D6B29200FFF7F8
:10154000A3FF95F82430A41B17441E449044E4B232
:10155000F6B2082E85F82460DBD1FFF721FF0028C2
:10156000D7D108E02B6A03EB82038342CFD0FFF789
:1015700017FF0028CBD10020BDE8F8830120FBE74E
:1015800080240020024B1A78024B1A70704700BF6B
:10159000C02400201022002038B51A4C1A4D2046D5
:1015A00001F01CFC2946204601F044FC2D68174838
:1015B000D5F89020D2F8043843F00203C2F804387A
:1015C00002F0B0FA2846124901F042FDD5F8902009
:1015D000104DD2F80438286823F002030E49A042C7
:1015E000C2F804384FF4E1330B6001D001F054FB32
:1015F0006868A04204D00849BDE8384001F04CBBFF
:1016000038BD00BF402B00207C64000840420F0022
:101610008464000814220020A82400200C4B70B51C
:101620000C4D04461E780C4B55F826209A420DD0DE
:101630000A4B002118221846FFF758FF04600146A4
:1016400055F82600BDE8704001F026BB70BD00BF14
:10165000C024002014220020402B0020A8240020B9
:1016600038B5084B04461546017543600A212430FD
:1016700002F07EFF04F128002A460A2102F078FFDA
:10168000204638BD50630008F8B51E461B68054665
:101690000C4617461BB9236863B9012408E0BDF85E
:1016A00018203146806A02F07BFF0028F3D1002425
:1016B0002046F8BD21463A46686A02F0A7FF044674
:1016C0000028EAD13368002BF1D0A86A02F0D2FFDB
:1016D000EEE7000038B50D46114604461A4611B132
:1016E000806A02F085FF2DB12946606ABDE8384066
:1016F00002F0B8BF38BD000070470000704700001E
:10170000002070470020704713B56C4600F11403A9
:1017100084E8060094E8030083E8050002B010BDE9
:101720000020704713B56C4600F10C0384E80600F6
:1017300094E8030083E8050002B010BD0023C0E96F
:101740000333704782B002AB03E9060002B0704772
:10175000704700000020704770470000002070476D
:10176000002070470120704782B0002002A901E9E3
:101770000C0002B070470000002070470020704746
:101780000B6883634B6843638B68C363CB680364F4
:101790000B6943647047000038B5036B0446154D70
:1017A0001B7955F8330001F04FFFD4E90B231B7967
:1017B00055F8331002F130034968994218D00023DC
:1017C0001363E26A5363D4E90B12537C581E137CF3
:1017D00092681B0443EA002313438B63D4E90B1381
:1017E0001B79303155F83300BDE8384001F0C0BEF8
:1017F00038BD00BFD8610008F8B51D4F05460E463C
:1018000011463868FFF75EFE78BB74683B7924B3F5
:1018100094F82C209A420BD02468F8E70122B521D5
:10182000FFF71EFF736823603B79746084F82C30E7
:10183000482004F0CDFB68B100220271C0E9032208
:10184000C0E90522027A42F007020272094AC0E9A1
:101850000B47026028602846F8BD402004F0B8FB22
:1018600004460028DAD12C60F5E700232B60F2E76C
:10187000C4240020E8610008044B10B5044603604E
:10188000406A08B104F0A2FB204610BD8C6100083C
:1018900010B50446FFF7F0FF204604F095FB204604
:1018A00010BD000008B519B1FFF776FF012008BD93
:1018B000036B1A79024B53F8320001F0C9FEF5E7C9
:1018C000D86100082DE9FF41DDF82880054617465C
:1018D00003911FFA88F60293FFF75EFF02ABBAB2DC
:1018E00003A9E86A0096FFF7CFFE044638B9002145
:1018F0002846FFF7D7FF204604B0BDE8F081AFB916
:101900002B6B05F134011A79134B53F83200B8F1FF
:10191000000F19D101F03AFE80F00104E4B2334621
:10192000E86ADDE90221FFF7D5FEE0E7029B83B913
:101930002B6B3A46084805F134011C79039B50F89B
:10194000340001F039FEE7E7029B424601F04AFE0F
:10195000E2E70024E3E700BFD861000813B50446BE
:101960000191FFF719FF019A236B04F134011879F3
:10197000054B53F8300001F04BFE00212046FFF7E5
:1019800091FF012002B010BDD861000810B50446D7
:10199000FFF702FF236B1A79054B53F8320001F071
:1019A00045FE00212046FFF77DFF012010BD00BF4E
:1019B000D8610008064B0121064A1A6000221A71FC
:1019C000054AC3E902124FF406721A82704700BF3B
:1019D000C424002078610008000E270700B59BB0E2
:1019E000EFF3098168226846FFF74EFDEFF30583A8
:1019F000014B9B6BFEE700BF00ED00E008B5FFF771
:101A0000EDFF000000B59BB0EFF309816822684646
:101A1000FFF73AFDEFF30583014B5B6BFEE700BF79
:101A200000ED00E0FEE70000FEE700000FB408B59F
:101A3000029802F007F8FEE702F0FCBC02F0D4BC0A
:101A400080697047C0697047006A7047406A704794
:101A5000806A7047F0B5ADF2044D0E460546002190
:101A60004FF47F7201A80091FFF740FD2C6A744388
:101A700001362B6A7343A34216D92B686A46214666
:101A800028465F684FF48063B84770B16A464FF4E8
:101A9000806312F8011BFF290AD1013B9BB2002B86
:101AA000F7D104F58064E4E701200DF2044DF0BDA8
:101AB0000020FAE780680368DB69184730B5456A9B
:101AC00085B004468D420FD30568CDE90023026A34
:101AD00003ABAD6A5143A84720B1206A039BC31AE8
:101AE0005842584105B030BD0020FBE7F0B5C5694C
:101AF00087B004468D4212D30C9F866905687143F6
:101B0000CDE9013705AB00936D69036AA84720B1A1
:101B1000A069059BC31A5842584107B0F0BD002088
:101B2000FBE70000F0B5662389B0002405464FF4BA
:101B300080768068079403A9CDE90336CDE9054492
:101B400003685B699847A8682246214603680094A9
:101B50001F692346B847A8689923079403A9CDE9CC
:101B60000336CDE9054403685B699847A8682246B7
:101B70002146036800941D692346A84709B0F0BDBB
:101B8000254B2DE9F04F1B789FB0002504468DF8BA
:101B900028304FF09F0E80684FF00123ADF8295098
:101BA00005A90995CDE905E3CDE9075503685B690A
:101BB0009847A06803222946036800922A461E69B6
:101BC0000AABB04728B394F88C20144B9DF828102A
:101BD00003EBC2031A7991421BD19DF829205B794E
:101BE0009A4216D1A0684FF05A0C0D4B082605A951
:101BF0000996CDE905C3CDE9075503685B699847A8
:101C0000A0682A462946036800961F690AABB847B0
:101C100040B9002048E100BFE8600008E862000821
:101C2000002500010422B1490AA804F001FA054682
:101C30000028EED1BDF82C306FF48277A3813B44AD
:101C4000012BE6D8079605A9CDE90A00A06803682C
:101C50005B699847A0682A462946036800961E6972
:101C60000AABB0470028D4D0DDE90A361A0202F4E4
:101C7000706242EA1662FF2ACBD11B0E26F07F4625
:101C800050222946142B26610AA828BF1423A373C7
:101C9000FFF72CFCA068079605A903685B699847C5
:101CA000A068A37B294602689B0000930AAB1669D3
:101CB0002A46B0470028ACD00B990029A9DBC908F7
:101CC0006FF07E43149D4FF0010E994228BF1946D4
:101CD000C5F303130EFA03F221FA03F303916161D2
:101CE000A261E361002B94D02646A44600274FF062
:101CF00002081EAAC7F3460302EB830353F834AC71
:101D000007F001031B01DA1D0EFA03F908FA02F2CB
:101D1000A2EB090202EA0A02DA401AD003F108092A
:101D20000F330EFA02F2216A08FA03F30EFA09FBE6
:101D3000CCF830208A42A3EB0B0B0BEA0A0A2AFAF2
:101D400009F98CF82C90A36A88BF2262934288BF5D
:101D5000A26201370CF1100C042FCAD1236A4FF094
:101D6000020C039A4FF0010E139F9A4224BFB2FB5C
:101D7000F3F1616207F00F0138BF01234FF0090250
:101D800001F1010138BF63624900336B33B3531C67
:101D90000EFA02F8A2F105090CFA03F30EFA09FA99
:101DA000A3EB080302F1FF380CFA08F83B40A8EB5C
:101DB0000A08D34008EA070828FA09F877D0012B67
:101DC00077D0022B77D0032B08BF4FF47A735FFADA
:101DD00088F808FB033373634B43B3630732103651
:101DE000252AD2D115F0C04FC5F3417365D0012B20
:101DF00065D0022B0CBF4FF47A634FF47A43C5F3DE
:101E0000046202FB0333E3664B432367199B9E077F
:101E100058D0062384F8743015F4005F05F00F03E2
:101E2000C5F3042514BF40220822013305FB022517
:101E30005B00A5675D430A9B9F02E5677FF5E9AEFE
:101E40000C9B1A0A84F88020C3F3421203F01F038C
:101E500084F8882084F88130189BC3F3025213F46D
:101E6000401F84F883207FF4D4AEDE0602D5042A16
:101E70007FF4CFAE03F40072002A14BF01220022C7
:101E800084F8872004D0DD0324D5002384F889302A
:101E9000179B1A0722D5002384F88630702384F814
:101EA0008530012384F88D301FB0BDE8F08F012309
:101EB0008DE710238BE7802389E710239FE74FF4FA
:101EC00080739CE7590701D55023A3E713F0780FDF
:101ED000A2D09EE69903DBD50123D7E75B07E0D5C7
:101EE000012384F886300523D9E700BF4862000843
:101EF00030B58BB000240546806803924FF0012274
:101F0000059105A9CDE90624CDE908440268526986
:101F10009047A8680121039B02680091214615693A
:101F20002246A8470BB030BD13B504460DF1070299
:101F300090F88510FFF7DCFF94F886309DF80700D5
:101F40001BB100F0010002B010BDC043C0F3C010CF
:101F5000F9E7000030B54FF001238BB000240546AF
:101F600080688DF80F20059105A9CDE90634CDE9EB
:101F7000084403685B699847A86801220DF10F01C6
:101F8000036800941D692346A8470BB030BD0000CC
:101F9000F7B517460DF1070206461D46FFF7A8FFE5
:101FA00068B19DF8074039469DF82020304624EA64
:101FB00005042A4022438DF80720FFF7CBFF03B02A
:101FC000F0BD000030B54FF4807389B000240546A1
:101FD0008068039103A9CDE90434CDE90644036880
:101FE0005B699847A86822462146036800941D69EA
:101FF0002346A84709B030BD10B5044623682046E3
:10200000DB6A98470028F9D110BD000010B590F8A0
:10201000743004465BB1FFF7EFFF012394F87410AE
:10202000204684F88E30BDE81040FFF7CBBF01207A
:1020300010BD000010B590F87430044653B1FFF79E
:10204000DBFF01232046042184F88E30BDE81040D8
:10205000FFF7B8BF012010BD70B590F883308AB08B
:102060000446042B48D10DF10E020521FFF740FF75
:1020700000282FD00DF10F0235212046FFF738FF41
:1020800040B320461E4EFFF7C1FF2046FFF7B4FFC6
:1020900005AD0FCE0FC5336805A99DF80E202B6046
:1020A0009DF80F30A06843F002038DF810208DF8E2
:1020B0000F308DF8113003685B699847A0680023E2
:1020C00004A90268009315690222A84728B920468E
:1020D000FFF7B0FF00200AB070BD2046FFF7AAFF4F
:1020E0000DF10F0235212046FFF702FF0028F1D045
:1020F0009DF80F309B07EDD501202071EBE700BF65
:10210000EC6000082DE9F341002304468068A360D9
:1021100010B103685B6898470025244E244F56F899
:10212000352001A839465FFA85F8FFF765FB019B6A
:10213000A0680022A360019210B103685B68984711
:10214000019810B103685B689847A368DBB141F25E
:10215000883084F88C8001F0E5FC2046FFF7E2FC33
:102160001E2001F0DFFC2046FFF70AFD054680B97E
:1021700094F88C300F4856F83310FFF781F9284651
:1021800002B0BDE8F0810135032DC8D10A48FFF740
:102190004DFC2046FFF760FF94F88C30054656F85A
:1021A000331008B90548E8E70548E6E7E8620008A3
:1021B000DC24002050620008C66200087A62000831
:1021C000A46200082DE9F041044688B00F46164687
:1021D000FFF71CFF2046FFF70FFF0025C722A0686E
:1021E0004FF48073079503A9CDE90323CDE9055585
:1021F00003685B699847A0682A46294603680095EA
:10220000D3F810802B46C047054630B92046FFF76B
:1022100011FF284608B0BDE8F081E36E3B60236FF4
:102220003360F3E72DE9F041002588B01F460446EE
:102230000E460E9B00F1400CA8463D60016B81B13B
:10224000A9420ED391420CD8B6FBF1FE01FB1E61F0
:1022500039B9416B90F82C800F9D1960816B296012
:10226000154610306045E9D16DB3AB1962699342F0
:1022700029D82046FFF7CAFE2046FFF7BDFE4FF4DF
:102280001453A06803A9CDF80C80CDE904360026CC
:10229000CDE9066603685B699847A0683246314617
:1022A00003680096D3F810803346C04706462046A0
:1022B0002EB9FFF7BFFE304608B0BDE8F081FFF74A
:1022C000B9FE3D60F7E70026F5E700002DE9F04193
:1022D0008669054688B00F46B3429046B1FBF6FCCE
:1022E00006FB1C1C28BF3346A6EB0C0C00269C45A5
:1022F000644628BF1C46FFF789FE2846FFF77CFE90
:102300000222A86803A9164B0597CDE90323CDE95E
:10231000066603685B699847A868224641460368D9
:1023200000961F693346B847064628462EB9FFF780
:1023300081FE304608B0BDE8F081FFF77BFE0E9BC2
:102340001C60AB6FAA696343B3FBF2F30F9A13608F
:10235000EA6F109B5443AA69B4FBF2F41C60E8E7EF
:10236000002500012DE9F04FCE18436989B00446DD
:102370009E420F46904634D83D464FF00009DFF8A4
:1023800070A0FFF739FEAE422FD9A6EB050B94F8EB
:10239000803094F8882003A9BBF5806F039394F8EC
:1023A000813028BF4FF4806B012AA06808BF03F179
:1023B000FF33CDF810A0CDE90559079303685B6999
:1023C0009847A068A8EB07030268CDF800B02B443B
:1023D000D2F810B000221146D84718B105F5806533
:1023E000D1E7002009B0BDE8F08F0120FAE700BF77
:1023F00000ED0003F0B5044689B00E46FFF7FCFD82
:1024000094F887502DB194F889302BB1012B1DD051
:102410000025284609B0F0BD94F880200392A5223B
:1024200006921A4ACDE9042394F88130A06803A9E2
:10243000079303685B699847A068314603689B6906
:1024400098470546642001F06DFBE2E7204600272F
:10245000FFF7DCFD2046FFF7CFFD08238122852111
:1024600020460097FFF794FD054618B92046FFF770
:10247000E1FDCEE794F8803006970393044BCDE955
:10248000043794F88130013BD0E700BF00ED000332
:1024900000ED0013014B024A1A607047DC24002053
:1024A0003C620008036800211B68184703790BB1E0
:1024B000002202711846704703685B6818470000E5
:1024C00003791BB901230371184670470020704738
:1024D0007047000010B5044603F076FD204610BD9D
:1024E00030B50A44084D91420DD011F8013B5840D7
:1024F000082340F30004013B2C4013F0FF0384EA5F
:102500005000F6D1EFE730BD2083B8ED38B58369D0
:1025100004460D465B695A0118D543681B682BB108
:102520000522027098472378052B01D102232370DE
:10253000202383F31188002104F1080001F00CFB33
:10254000002383F31188E06902F03AFAEB0704D51F
:102550000248BDE8384001F075BA38BD686300082C
:1025600010B5044C204600F0FBFF034A0023C4E9E9
:10257000062310BDE42400200050005210B503785B
:102580000446012B17D1104B984214D102460F4933
:10259000102002F0E1F90E4BE061D3F8D42042F4B0
:1025A0008042C3F8D420D3F8FC2042F48042C3F820
:1025B000FC20D3F8FC306268A36992685A60054A2F
:1025C0001A601B22DA6010BDE42400200D250008EB
:1025D000004402581500020183691B2210B5DA601D
:1025E000D1E9002012F44C4406D192011C61D8615B
:1025F00002F440425A6110BD0024104312F4406FAF
:102600001C61CC68DC61586101D08A689A619A6863
:102610009206FCD4EFE7000030B584691B25C06941
:10262000E5600068836104F12003C3610223426115
:10263000013A03614623C36016238362CB6822619B
:10264000E361D1E90023134312F4406F636101D0C9
:102650008B68A361C36843F00103C36030BD000011
:1026600030B5D0E90640006804F120058561C361FA
:1026700008234261013A036146230D69C3601623B2
:102680008362CB682261E361D1E90023134312F432
:10269000406F43EA854343F08063636101D08B68F8
:1026A000A361C36843F00103C36030BD8069036860
:1026B00023F0040310B5036000230361C361836149
:1026C000D1E900430969234343EA814343F040636E
:1026D000436112B14FF01043136010BD83691A6853
:1026E00042F002021A601A689207FCD41A6842F09B
:1026F00004021A607047000083691B2210B5DA607B
:1027000004465B695B011AD443681B682BB1052240
:10271000027098472378052B01D1022323702023D0
:1027200083F31188002104F1080001F015FA002359
:1027300083F31188E069BDE8104002F041B910BD93
:10274000026843681143016003B1184770470000F5
:10275000024A136843F0C003136070470010014041
:1027600013B50E4C204600F08BFA04F11400002340
:102770004FF400720A49009400F04CF9094B4FF4F1
:102780000072094904F13800009400F0C5F9074AC5
:10279000074BC4E9172302B010BD00BF0425002079
:1027A00070250020512700087027002000100140EC
:1027B00000E1F505037C30B5244C002918BF0C4618
:1027C000012B11D1224B98420ED1224BD3F8F0208D
:1027D00042F01002C3F8F020D3F8182142F01002A2
:1027E000C3F81821D3F818312268036EC16D03EBCA
:1027F00052038466B3FBF2F36268150442BF23F010
:10280000070503F0070343EA4503CB60A36843F0E1
:1028100040034B60E36843F001038B6042F496731E
:1028200043F001030B604FF0FF330B62510505D5F8
:1028300012F0102205D0B2F1805F04D080F864302D
:1028400030BD7F23FAE73F23F8E700BF7863000835
:1028500004250020004402582DE9F047C66D0546C6
:102860003768F4692107346219D014F0080118BFE1
:102870008021E20748BF41F02001A3074FF0200369
:1028800048BF41F04001600748BF41F4807183F3C5
:102890001188281DFFF754FF002383F31188E205F8
:1028A0000AD5202383F311884FF40071281DFFF708
:1028B00047FF002383F311884FF020094FF0000AEF
:1028C00014F0200838D13B0616D54FF0200905F149
:1028D000380A200610D589F31188504600F050F9C7
:1028E000002836DA0821281DFFF72AFF27F0800389
:1028F0003360002383F31188790614D5620612D55C
:10290000202383F31188D5E913239A4208D12B6C35
:1029100033B127F040071021281DFFF711FF376062
:10292000002383F31188E30618D5AA6E1369ABB1AF
:102930005069BDE8F047184789F31188736A284643
:1029400095F86410194000F0B5F98AF31188F4691C
:10295000B6E7B06288F31188F469BAE7BDE8F0879A
:10296000F8B51546826804460B46AA4200D285682F
:10297000A1692669761AB5420BD218462A46FEF797
:1029800083FDA3692B44A3612846A3685B1BA36056
:10299000F8BD0CD9AF1B18463246FEF775FD3A4616
:1029A000E1683044FEF770FDE3683B44EBE718460E
:1029B0002A46FEF769FDE368E5E700008368934275
:1029C000F7B50446154600D28568D4E90460361A86
:1029D000B5420BD22A46FEF757FD63692B4463616B
:1029E0002846A3685B1BA36003B0F0BD0DD9324637
:1029F000AF1B0191FEF748FD01993A46E06831446A
:102A0000FEF742FDE3683B44E9E72A46FEF73CFD5A
:102A1000E368E4E710B50A440024C361029B8460C4
:102A2000C16002610362C0E90000C0E9051110BD88
:102A300008B5D0E90532934201D1826882B9826833
:102A4000013282605A1C426119700021D0E90432BF
:102A50009A4224BFC368436101F098F8002008BD82
:102A60004FF0FF30FBE7000070B5202304460E4610
:102A700083F31188A568A5B1A368A269013BA3608F
:102A8000531CA36115782269934224BFE368A361B4
:102A9000E3690BB120469847002383F31188284649
:102AA00007E03146204601F061F80028E2DA85F3BC
:102AB000118870BD2DE9F74F04460E46174698461B
:102AC000D0F81C904FF0200A8AF311884FF0000BC9
:102AD000154665B12A4631462046FFF741FF0346B9
:102AE00060B94146204601F041F80028F1D00023AA
:102AF00083F31188781B03B0BDE8F08FB9F1000FA4
:102B000003D001902046C847019B8BF31188ED1A32
:102B10001E448AF31188DCE7C160C361009B8260B8
:102B20000362C0E905111144C0E90000016170476A
:102B3000F8B504460D461646202383F31188A7688E
:102B4000A7B1A368013BA36063695A1C62611D7051
:102B5000D4E904329A4224BFE3686361E3690BB1AC
:102B600020469847002080F3118807E03146204630
:102B700000F0FCFF0028E2DA87F31188F8BD0000BE
:102B8000D0E9052310B59A4201D182687AB98268EA
:102B90000021013282605A1C82611C7803699A42CA
:102BA00024BFC368836100F0F1FF204610BD4FF0E1
:102BB000FF30FBE72DE9F74F04460E4617469846CF
:102BC000D0F81C904FF0200A8AF311884FF0000BC8
:102BD000154665B12A4631462046FFF7EFFE03460B
:102BE00060B94146204600F0C1FF0028F1D0002323
:102BF00083F31188781B03B0BDE8F08FB9F1000FA3
:102C000003D001902046C847019B8BF31188ED1A31
:102C10001E448AF31188DCE70268436811430160AF
:102C200003B11847704700001430FFF743BF00009E
:102C30004FF0FF331430FFF73DBF00003830FFF78F
:102C4000B9BF00004FF0FF333830FFF7B3BF0000CB
:102C50001430FFF709BF00004FF0FF311430FFF7C9
:102C600003BF00003830FFF763BF00004FF0FF32B2
:102C70003830FFF75DBF000000207047FFF770BDE0
:102C8000044B036000234360C0E902330123037453
:102C9000704700BF9063000810B52023044683F3FB
:102CA0001188FFF787FD02232374002383F3118823
:102CB00010BD000038B5C36904460D461BB9042198
:102CC0000844FFF7A9FF294604F11400FFF7B0FEFE
:102CD000002806DA201D4FF48061BDE83840FFF778
:102CE0009BBF38BD026843681143016003B11847B8
:102CF0007047000013B5406B00F58054D4F8A43839
:102D00001A681178042914D1017C022911D119798A
:102D1000012312898B4013420BD101A94C3002F0E0
:102D20009BFCD4F8A4480246019B2179206800F05E
:102D3000DFF902B010BD0000143002F01DBC00002D
:102D40004FF0FF33143002F017BC00004C3002F09B
:102D5000EFBC00004FF0FF334C3002F0E9BC000044
:102D6000143002F0EBBB00004FF0FF31143002F0E2
:102D7000E5BB00004C3002F0BBBC00004FF0FF325E
:102D80004C3002F0B5BC00000020704710B500F5D3
:102D90008054D4F8A4381A681178042917D1017C1A
:102DA000022914D15979012352898B4013420ED143
:102DB000143002F07DFB024648B1D4F8A4484FF429
:102DC000407361792068BDE8104000F07FB910BD04
:102DD000406BFFF7DBBF0000704700007FB5124B70
:102DE00001250426044603600023057400F18402D3
:102DF00043602946C0E902330C4B02901430019322
:102E00004FF44073009602F02FFB094B04F69442F6
:102E1000294604F14C000294CDE900634FF440735D
:102E200002F0F6FB04B070BDB8630008D12D0008B5
:102E3000F52C00080A68202383F311880B790B33E3
:102E400042F823004B79133342F823008B7913B1F6
:102E50000B3342F8230000F58053C3F8A418022373
:102E60000374002383F311887047000038B5037F93
:102E7000044613B190F85430ABB90125201D02214E
:102E8000FFF730FF04F114006FF00101257700F027
:102E900089FE04F14C0084F854506FF00101BDE844
:102EA000384000F07FBE38BD10B501210446043023
:102EB000FFF718FF0023237784F8543010BD00007B
:102EC00038B504460025143002F0E6FA04F14C004F
:102ED000257702F0B5FB201D84F854500121FFF73F
:102EE00001FF2046BDE83840FFF750BF90F8803022
:102EF00003F06003202B06D190F881200023212AC3
:102F000003D81F2A06D800207047222AFBD1C0E927
:102F10001D3303E0034A426707228267C36701202B
:102F2000704700BF3422002037B500F58055D5F832
:102F3000A4381A68117804291AD1017C022917D102
:102F40001979012312898B40134211D100F14C04ED
:102F5000204602F035FC58B101A9204602F07CFB66
:102F6000D5F8A4480246019B2179206800F0C0F8FA
:102F700003B030BD01F10B03F0B550F8236085B00C
:102F800004460D46FEB1202383F3118804EB850728
:102F9000301D0821FFF7A6FEFB6806F14C005B69B7
:102FA0001B681BB1019002F065FB019803A902F0B8
:102FB00053FB024648B1039B2946204600F098F88F
:102FC000002383F3118805B0F0BDFB685A691268CD
:102FD000002AF5D01B8A013B1340F1D104F1800295
:102FE000EAE70000133138B550F82140ECB1202356
:102FF00083F3118804F58053D3F8A4281368527919
:1030000003EB8203DB689B695D6845B104216018AE
:10301000FFF768FE294604F1140002F053FA204637
:10302000FFF7B4FE002383F3118838BD704700001A
:1030300001F046BD01234022002110B5044600F8EE
:10304000303BFEF753FA0023C4E9013310BD000002
:1030500010B52023044683F3118824224160002107
:103060000C30FEF743FA204601F04CFD022323709A
:10307000002383F3118810BD70B500EB8103054672
:1030800050690E461446DA6018B110220021FEF78E
:103090002DFAA06918B110220021FEF727FA314657
:1030A0002846BDE8704001F03FBE00008368202242
:1030B000002103F0011310B5044683601030FEF7C1
:1030C00015FA2046BDE8104001F0BABEF0B4012563
:1030D00000EB810447898D40E4683D43A469458144
:1030E00023600023A2606360F0BC01F0D7BE000043
:1030F000F0B4012500EB810407898D40E4683D436D
:103100006469058123600023A2606360F0BC01F064
:103110004DBF000070B50223002504462422037031
:103120002946C0F888500C3040F8045CFEF7DEF900
:10313000204684F8705001F08BFD63681B6823B152
:1031400029462046BDE87040184770BD037880F8D6
:103150008C300523037043681B6810B504460BB11F
:10316000042198470023A36010BD000090F88C2034
:10317000436802701B680BB10521184770470000B7
:1031800070B590F87030044613B1002380F87030A9
:1031900004F18002204601F077FE63689B68B3B9B2
:1031A00094F8803013F0600535D00021204602F0FD
:1031B00021F90021204602F011F963681B6813B160
:1031C000062120469847062384F8703070BD2046BB
:1031D00098470028E4D0B4F88630A26F9A4288BF9E
:1031E000A36794F98030A56F002B4FF0200380F285
:1031F0000381002D00F0F280092284F8702083F30F
:10320000118800212046D4E91D23FFF771FF002318
:1032100083F31188DAE794F8812003F07F0343EA0F
:10322000022340F20232934200F0C58021D8B3F568
:10323000807F48D00DD8012B3FD0022B00F0938027
:10324000002BB2D104F1880262670222A267E36711
:10325000C1E7B3F5817F00F09B80B3F5407FA4D137
:1032600094F88230012BA0D1B4F8883043F00203E7
:1032700032E0B3F5006F4DD017D8B3F5A06F31D061
:10328000A3F5C063012B90D86368204694F8822090
:103290005E6894F88310B4F88430B047002884D076
:1032A000436863670368A3671AE0B3F5106F36D00D
:1032B00040F6024293427FF478AF5C4B636702238F
:1032C000A3670023C3E794F88230012B7FF46DAF2E
:1032D000B4F8883023F00203A4F88830C4E91D55FF
:1032E000E56778E7B4F88030B3F5A06F0ED194F8B5
:1032F0008230204684F88A3001F008FD63681B683C
:1033000013B1012120469847032323700023C4E909
:103310001D339CE704F18B0363670123C3E7237824
:10332000042B10D1202383F311882046FFF7BEFE23
:1033300085F311880321636884F88B5021701B6822
:103340000BB12046984794F88230002BDED084F8E9
:103350008B300423237063681B68002BD6D00221B6
:1033600020469847D2E794F8843020461D0603F0A3
:103370000F010AD501F07AFD012804D002287FF45C
:1033800014AF2B4B9AE72B4B98E701F061FDF3E765
:1033900094F88230002B7FF408AF94F8843013F057
:1033A0000F01B3D01A06204602D502F03BF8ADE774
:1033B00002F02CF8AAE794F88230002B7FF4F5AEE7
:1033C00094F8843013F00F01A0D01B06204602D5DC
:1033D00002F010F89AE702F001F897E7142284F857
:1033E000702083F311882B462A4629462046FFF792
:1033F0006DFE85F31188E9E65DB1152284F8702031
:1034000083F3118800212046D4E91D23FFF75EFED7
:10341000FDE60B2284F8702083F311882B462A46A0
:1034200029462046FFF764FEE3E700BFE863000893
:10343000E0630008E463000838B590F87030044693
:10344000002B3ED0063BDAB20F2A34D80F2B32D8ED
:10345000DFE803F037313108223231313131313197
:1034600031313737856FB0F886309D4214D2C3684A
:103470001B8AB5FBF3F203FB12556DB9202383F3CE
:1034800011882B462A462946FFF732FE85F311881C
:103490000A2384F870300EE0142384F8703020235F
:1034A00083F31188002320461A461946FFF70EFEC3
:1034B000002383F3118838BDC36F03B198470023FD
:1034C000E7E70021204601F095FF0021204601F0AA
:1034D00085FF63681B6813B10621204698470623C1
:1034E000D7E7000010B590F870300446142B29D0AF
:1034F00017D8062B05D001D81BB110BD093B022BF4
:10350000FBD80021204601F075FF0021204601F084
:1035100065FF63681B6813B10621204698470623A0
:1035200019E0152BE9D10B2380F87030202383F3A9
:10353000118800231A461946FFF7DAFD002383F3AA
:103540001188DAE7C3689B695B68002BD5D1C36F2C
:1035500003B19847002384F87030CEE7FFF700B836
:10356000012100230170C0E901330C3000F008BADA
:1035700010B52023044683F311884160FEF7FEFF57
:1035800002232370002383F3118810BD10B520237C
:10359000044683F31188032304F8083BFFF71CF863
:1035A0004FF0FF31204600F0C9FA002383F3118861
:1035B000C01A18BF012010BD38B50446202585F378
:1035C0001188032504F8085BFFF726F84FF0FF3158
:1035D000204600F0B3FA002383F31188C01A18BF05
:1035E000012038BD38B50446202585F3118804250F
:1035F00004F8085BFFF734F84FF0FF31204600F085
:103600009DFA002383F31188C01A18BF012038BD2A
:1036100010B52023044683F31188FFF747F80623EB
:103620002370002383F3118810BD000010B5202300
:10363000044683F31188FFF751F802232370002317
:1036400083F3118810BD00000C3000F0B5B9000004
:103650000C3000F0BBB9000004480121044B0360AA
:103660000023C0E901330C3000F08AB97029002032
:1036700075580008CB1D083A23F00703591A521A4F
:10368000012110B4D2080024C0E9004384600C304A
:103690001C605A605DF8044B00F072B92DE9F84FD8
:1036A000364ECD1D0F46002818BF0646082A4FEAA1
:1036B000D50538BF082206F10C08341D9146404656
:1036C00000F07AF909F10701C9F1000E22462468D9
:1036D0006CB9404600F07AF93368CBB3082249460A
:1036E000E8009847044698B340E9026730E004EBED
:1036F000010CD4F804A00CEA0E0C0AF10100ACF1A4
:10370000080304EBC0009842E0D9A0EB0C0CB5EB29
:10371000EC0F4FEAEC0BD9D89C421CD204F1080202
:10372000AB45A3EB02024FEAE202626009D9691CD1
:10373000ED43206803EBC1025D44556043F831005E
:1037400022601C465F60404644F8086B00F03EF97A
:103750002046BDE8F88FAA45216802D111602346B2
:10376000EFE7013504EBC50344F8351003F1080118
:10377000401AC01058601360F1E700BF70290020A4
:10378000F8B550F8043C044650F8085CA0F108066F
:1037900007332F1D0C35DB0840F8043C284600F0A9
:1037A0000BF93B46BB421A6801D09E4228D90AB1A8
:1037B000964225D244F8082C54F8042C1E6001329D
:1037C00054F8081C06EBC200814206D14868024446
:1037D00044F8042C0A6844F8082C5868411C03EB90
:1037E000C1018E4207D154F8042C013202445A60C0
:1037F00054F8082C1A602846BDE8F84000F0E6B8F6
:103800001346CFE7024B0022C3E900339A607047AA
:1038100088290020002382680374054B1B6899687F
:103820009142FBD25A680360426010605860704752
:103830008829002008B5202383F31188027C002307
:10384000052A06D8DFE802F00B050503120E4269CF
:1038500013604FF0FF334361FFF7DCFF002383F376
:10386000118808BD4269936801339360D0E9003242
:1038700013605A60EDE70000002382680374054B73
:103880001B6899689142FBD85A68036042601060D7
:103890005860704788290020054B1969087418681A
:1038A000026853601A60186101230374FCF718BFA3
:1038B000882900204B1C30B5044687B00A4D10D033
:1038C0002B6901A8094A00F089F92046FFF7E4FFB7
:1038D000049B13B101A800F0BDF92B69586907B02A
:1038E00030BDFFF7D9FFF8E78829002035380008F8
:1038F00038B50C4D044641612B6981689A68914244
:1039000003D8BDE83840FFF785BF1846FFF7B4FF7E
:1039100001232C61014623742046BDE83840FCF7A2
:10392000DFBE00BF88290020044B1A681B6990681D
:103930009B68984294BF002001207047882900208E
:1039400010B5084C236820691A685460226001226F
:1039500023611A74FFF790FF01462069BDE810400B
:10396000FCF7BEBE8829002008B5FFF7DDFF18B1BF
:10397000BDE80840FFF7E4BF08BD0000FFF7E0BF67
:10398000C0E90000816070478368013B002B10B5DF
:1039900083600DDA074C42682369586118605A60E9
:1039A000136043600520FFF777FF2369586910BD56
:1039B0000020FCE78829002008B5202383F3118824
:1039C000FFF7E2FF002383F3118808BD08B5202329
:1039D00083F3118883680133002B836007DC03685D
:1039E00000211A68026050601846FFF781FF00232B
:1039F00083F3118808BD0000FEE7000010B50E4CEF
:103A0000FFF700FF00F0DCF801F016FFFFF724FEDF
:103A100080220A49204600F047F8012344F8180C98
:103A2000037400F051FE002383F3118862B604484A
:103A3000BDE8104000F058B8B0290020EC63000841
:103A4000FC63000808B572B6034B586200F0BEFC78
:103A500000F08CFDFEE700BF8829002000F034B99B
:103A6000EFF3118020B9EFF30583202282F3118850
:103A70007047000010B530B9EFF30584C4F30804B3
:103A800014B180F3118810BDFFF76EFF84F3118825
:103A9000F9E70000034A516853685B1A9842FBD863
:103AA000704700BF001000E082600222028270476F
:103AB0008368A3F17C0243F80C2C026943F83C2C88
:103AC000426943F8382C074A43F81C2CC268A3F11A
:103AD000180043F8102C022203F8082C002203F8E7
:103AE000072C7047F906000810B5202383F31188CE
:103AF000FFF7DEFF00210446FFF7FAFE002383F301
:103B00001188204610BD0000024B1B6958610F2030
:103B1000FFF7C2BE88290020202383F31188FFF716
:103B2000F3BF000008B50146202383F31188082065
:103B3000FFF7C0FE002383F3118808BD054B1B6906
:103B400021B1036058610320FFF7B4BE4FF0FF308E
:103B5000704700BF8829002003682BB10022026053
:103B600018465961FFF756BE7047000049B1064B31
:103B700042681B6918605A60136043600420FFF7B5
:103B800099BE4FF0FF3070478829002003689842A3
:103B900006D01A680260506018465961FFF73ABEB5
:103BA0007047000038B504460D462068844200D1B5
:103BB00038BD036823605C604561FFF72BFEF4E7C6
:103BC000054B4FF0FF3103F11402C3E90522002237
:103BD000C3E90712704700BF8829002070B51C4E4A
:103BE00005460C46C0E9032301F020FE334653F896
:103BF000142F9A420DD130620A2C2CBF00190A30C2
:103C00002A60C5E90124C6E90555BDE8704001F008
:103C1000F7BD316A431AE31838BF1C469368A342C4
:103C200002D9081901F0FCFD73699A6894420CD816
:103C30005A68AC602B606A6015609A685D60121B00
:103C40009A604FF0FF33F36170BDA41A1B68ECE774
:103C50008829002038B51B4C636998420DD08168D3
:103C6000D0E9003213605A600022C2609A680A44A8
:103C70009A604FF0FF33E36138BD036822460021AC
:103C800042F8143F93425A60C16003D1BDE8384006
:103C900001F0C0BD9A688168256A0A449A6001F003
:103CA000C5FD6369411B9A688A42E5D9AB181D1AA4
:103CB000206A092D98BF01F10A02BDE8384010447E
:103CC00001F0AEBD882900202DE9F041184C0027F5
:103CD00004F11406656901F0A9FD236AAA68C11AF6
:103CE0008A4215D81344D5F80C802362D5E90032F6
:103CF00013605A606369EF60B34201D101F08AFD3D
:103D000087F311882869C047202383F31188E1E7EE
:103D10006169B14209D013441B1ABDE8F0410A2B76
:103D20002CBFC0180A3001F07BBDBDE8F08100BF98
:103D30008829002000207047FEE70000704700003F
:103D40004FF0FF307047000002290CD0032904D047
:103D50000129074818BF00207047032A05D80548E5
:103D600000EBC2007047044870470020704700BF56
:103D7000E0640008442200209464000870B59AB002
:103D800005460846144601A900F0C2F801A8FDF74F
:103D9000A5FB431C0022C6B25B001046C5E90034F7
:103DA00023700323023404F8013C01ABD1B2023486
:103DB0008E4201D81AB070BD13F8011B013204F80D
:103DC000010C04F8021CF1E708B5202383F31188E5
:103DD0000348FFF7A9F8002383F3118808BD00BF4B
:103DE000402B002090F8803003F01F02012A07D1F9
:103DF00090F881200B2A03D10023C0E91D3315E080
:103E000003F06003202B08D1B0F884302BB990F870
:103E10008120212A03D81F2A04D8FFF767B8222A55
:103E2000EBD0FAE7034A426707228267C3670120A3
:103E3000704700BF3B22002007B5052917D8DFE8EF
:103E400001F0191603191920202383F31188104A51
:103E500001210190FFF710F9019802210D4AFFF7A7
:103E60000BF90D48FFF72CF8002383F3118803B0FA
:103E70005DF804FB202383F311880748FEF7F6FF63
:103E8000F2E7202383F311880348FFF70DF8EBE7EF
:103E90003464000858640008402B002038B50C4DED
:103EA0000C4C2A460C4904F10800FFF767FF05F1A6
:103EB000CA0204F110000949FFF760FF05F5CA7254
:103EC00004F118000649BDE83840FFF757BF00BFAE
:103ED0001844002044220020146400081E640008D6
:103EE0002964000870B5044608460D46FDF7F6FA49
:103EF000C6B22046013403780BB9184670BD32466D
:103F00002946FDF7CBFA0028F3D10120F6E700009F
:103F10002DE9F84F05460C46FDF7E0FA2C49C6B2EC
:103F20002846FFF7DFFF08B10336F6B229492846D5
:103F3000FFF7D8FF08B11036F6B2632E0DD8DFF8C0
:103F40009080DFF89090244FDFF894A0DFF894B0D1
:103F50002E7846B92670BDE8F88F29462046BDE880
:103F6000F84F02F0B9B8252E2ED107224146284637
:103F7000FDF794FA70B9DBF8003007350A3444F8DD
:103F80000A3CDBF8043044F8063CBBF8083024F85F
:103F9000023CDDE7082249462846FDF77FFA98B93A
:103FA000A21C0E4B197802320909C95D02F8041CE3
:103FB00013F8011B01F00F015345C95D02F8031C02
:103FC000F0D118340835C3E7013504F8016BBFE7B9
:103FD00000650008296400081365000800E8F11F67
:103FE0000CE8F11F08650008BFF34F8F044B1A69F6
:103FF0005107FCD1D3F810215207F8D1704700BF08
:104000000020005208B50D4B1B78ABB9FFF7ECFF51
:104010000B4BDA68D10704D50A4A5A6002F188329C
:104020005A60D3F80C21D20706D5064AC3F80421FA
:1040300002F18832C3F8042108BD00BF7646002093
:1040400000200052230167454FF00063054A1968BC
:10405000013104D104339342F9D10120704700208B
:10406000704700BF0000020808B5114B1B78F3B978
:10407000104B1A69510703D5DA6842F04002DA6042
:10408000D3F81021520705D5D3F80C2142F0400295
:10409000C3F80C21FFF7A8FF064BDA6842F00102D3
:1040A000DA60D3F80C2142F00102C3F80C2108BDFC
:1040B00076460020002000524FF400307047000088
:1040C0000120704708B9FFF7BFBF0020704700000C
:1040D00038B548BB154CFFF7C3FCFFF785FF054615
:1040E000FFF790FF4FF0FF336361C4F81431236191
:1040F000FFF77AFF2423E360E36843F08003E36083
:1041000023695B07FCD4FFF76FFF4FF000604FF4AB
:10411000003100F007FA2846FFF7A6FFFFF7AAFCD8
:10412000BDE83840FFF790BF002038BD00200052A6
:104130002DE9F84F40EA020305460C461746D8061B
:1041400002D00020BDE8F88F27F01F07DFF8D4B0B9
:10415000FFF758FF2744BC4203D10120FFF784FF3B
:10416000F0E720222946204601F062FF10B92035F1
:104170002034F0E72B4605F120021E68711CE0D1C7
:1041800004339A42F9D1FFF76BFC05F17843234AD7
:10419000B3F5801F224B28BF9A4603F1040338BFB2
:1041A0009046A2F1080228BF9846A3F108033ABF3F
:1041B0009146DA469946FFF717FFC8F80060A5EB6D
:1041C000040CD9F8002004F11C0142F00202C9F8E5
:1041D0000020221FDAF8006016F00506FAD152F826
:1041E000043F8A424CF80230F4D1BFF34F8FFFF7FF
:1041F000FBFE4FF0FF32C8F80020D9F8002022F073
:104200000202C9F80020FFF735FC2022214628468B
:1042100001F00EFF0028AAD030469FE7142000527C
:10422000102100521020005210B5084C237828B1FC
:104230001BB9FFF7E7FE0123237010BD002BFCD054
:104240002070BDE81040FFF70FBF00BF764600208A
:104250002DE9F74F0E460546002864D011F00507FA
:1042600063D139B9082229463046FFF717FA0446C8
:10427000002848D108224FF00109DFF8C08006F07D
:104280000403DFF8BCA006EA090BBBF1000F27D03E
:10429000D8F81410C80723D409F1010908F10C0853
:1042A000B9F1060FF1D18FB9224E2946F0190092CB
:1042B000FFF7F4F9044630BB1837009A782FF4D191
:1042C0002946FFF7EBF90446E8B9009A29461A484F
:1042D000FFF7E4F9044608BB204603B0BDE8F08FC1
:1042E000ABB1D8F8141011F0040FD5D0182029461E
:1042F00000FB09A0CDE90023FFF7D0F90446DDE972
:1043000000230028C8D02A460021204608E0B10733
:10431000ECD5D8F8141011F0020FE6E72A46002178
:10432000FDF7E4F8D8E70446D6E71F35202225F04C
:104330001F05A0E7A8460020784600202465000855
:10434000904600200021FFF783BF00000121FFF706
:104350007FBF0000F8B5144D01241827134E40F21A
:10436000FF3200210120FDF7C1F807FB0460013492
:104370002A6955F80C1FFFF77DF9062CF5D1372572
:104380004FF4C0542046FFF7E1FF014628B1224612
:104390000748BDE8F840FFF76DB9C4EBC404013D20
:1043A0004FEAD404EED1F8BD246500089046002001
:1043B000784600200421FFF74BBF00004843FFF779
:1043C000C1BF000008B1FFF7DBB9704738B5054D34
:1043D00000240334696855F80C0B00F0B5F8122C72
:1043E000F7D138BD2465000870B5104E82B0FFF7D4
:1043F00037FB054601F01AFA3268034690423360F3
:1044000037BF0B4A0A495168146836BF0131D1E9F8
:10441000004151600419284641F100010191FFF764
:1044200029FB2046019902B070BD00BF2047002043
:104430002847002070B5124E82B0FFF711FB0546E9
:1044400001F0F4F9326803469042336037BF0D4AF9
:104450000C495168146836BF0131D1E900415160FF
:104460000419284641F100010191FFF703FB4FF4C5
:104470007A72002320460199FBF71AFF02B070BD43
:1044800020470020284700200244074BD2B210B535
:10449000904200D110BD441C00B253F8200041F8F6
:1044A000040BE0B2F4E700BF504000580E4B30B5AB
:1044B0001C6F240405D41C6F1C671C6F44F400445B
:1044C0001C670A4C02442368D2B243F48073236011
:1044D000074B904200D130BD441C51F8045B00B240
:1044E00043F82050E0B2F4E7004402580048025874
:1044F0005040005807B5012201A90020FFF7C4FF72
:10450000019803B05DF804FB13B50446FFF7F2FF12
:10451000A04205D0012201A900200194FFF7C6FFA7
:1045200002B010BD0144BFF34F8F064B884204D345
:10453000BFF34F8FBFF36F8F7047C3F85C0220301B
:10454000F4E700BF00ED00E00144BFF34F8F064BDE
:10455000884204D3BFF34F8FBFF36F8F7047C3F808
:1045600070022030F4E700BF00ED00E0704700006B
:1045700070B5054616460C4601201021FFF71EFFB8
:10458000286046733CB1204636B1FFF713FF2B6815
:10459000186000B19C6070BDFFF7D8FEF7E700001F
:1045A00070B50E461546044600B30B684360836839
:1045B000934210D213B10068FFF704FF637B2846D3
:1045C0002BB1FFF7F7FE206020B9A06070BDFFF7A8
:1045D000BDFEF8E7A560206805F11F01306021F0FD
:1045E0001F01FFF79FFF01202073EFE70120EDE798
:1045F00010B5044640B10068884205D1606808B132
:10460000FCF742FF0023237310BD000070B50E4677
:104610001546044620B38368934210D213B1006854
:10462000FFF7D0FE637B28462BB1FFF7C3FE206067
:1046300020B9A06070BDFFF789FEF8E7A56031687A
:1046400019B12A462068FCF71FFF206805F11F01F9
:10465000306021F01F01FFF777FF01202073E9E7A9
:104660000120E7E720B103688B4204BF00230373F6
:104670007047000008B1002303737047034B1A68AA
:104680001AB9034AD2F8D0241A6070473047002084
:104690000040025808B5FFF7F1FF024B1868C0F35D
:1046A000806008BD30470020EFF309830549683377
:1046B0004A6B22F001024A6383F30988002383F3E3
:1046C0001188704700EF00E0202080F3118862B667
:1046D0000D4B0E4AD96821F4E0610904090C0A4324
:1046E0000B49DA60D3F8FC2042F08072C3F8FC205A
:1046F000084AC2F8B01F116841F001011160102290
:10470000DA7783F82200704700ED00E00003FA0535
:1047100055CEACC5001000E0202310B583F31188FE
:104720000E4B5B6813F4006314D0F1EE103AEFF314
:1047300009844FF08073683CE361094BDB6B2366AF
:1047400084F30988FFF7F0F810B1064BA36110BDA0
:10475000054BFBE783F31188F9E700BF00ED00E0AC
:1047600000EF00E00B0700080E07000870B5BFF36C
:104770004F8FBFF36F8F1A4A0021C2F85012BFF358
:104780004F8FBFF36F8F536943F400335361BFF30F
:104790004F8FBFF36F8FC2F88410BFF34F8FD2F8E3
:1047A000803043F6E074C3F3C900C3F34E335B01BA
:1047B00003EA0406014646EA81750139C2F86052EF
:1047C000F9D2203B13F1200FF2D1BFF34F8F536981
:1047D00043F480335361BFF34F8FBFF36F8F70BDCE
:1047E00000ED00E0FEE700000A4B0B480B4A904248
:1047F0000BD30B4BC11EDA1C121A22F003028B42A0
:1048000038BF00220021FCF771BE53F8041B40F8AA
:10481000041BECE7F0670008D8490020D8490020C5
:10482000D849002070470000036819685960436840
:104830000BB18068184770474FF0A44310B51C684F
:10484000E00702D52848FFF7EFFFA10702D5274868
:10485000FFF7EAFF620702D52548FFF7E5FF2307C8
:1048600002D52448FFF7E0FFE00602D52248FFF713
:10487000DBFFA10602D52148FFF7D6FF620602D56D
:104880001F48FFF7D1FF230602D51E48FFF7CCFFD4
:10489000E00502D51C48FFF7C7FFA10502D51B485C
:1048A000FFF7C2FF620502D51948FFF7BDFF2305D8
:1048B00002D51848FFF7B8FFE00402D51648FFF705
:1048C000B3FFA10402D51548FFF7AEFF620402D57D
:1048D0001348FFF7A9FF230402D51248FFF7A4FFEE
:1048E000BDE81040FFF718BF3847002044470020BC
:1048F000504700205C470020684700207447002094
:10490000804700208C47002098470020A4470020C3
:10491000B0470020BC470020C8470020D4470020F3
:10492000E0470020EC47002030B5094B0021094C3E
:1049300010200725196054F8042B0138C3E9012120
:10494000D16003F10C0311615560F4D130BD00BF9B
:10495000344700206C6500080F28F0B50AD91028EC
:1049600006D10F230020144C01272568984203D953
:1049700000201DE00346F6E707FA00F6354218D19D
:104980000C23354343432560181D2344C3E9021219
:104990000A4B2044D3F8D42042F00102C3F8D420BB
:1049A000D3F8FC2042F00102C3F8FC20D3F8FC301D
:1049B000F0BD0130DAE700BF344700200044025860
:1049C0000368D968DA68C90722F03F02DA6002D5C5
:1049D0001A689207FCD507225A60704770B5D0E973
:1049E000244300224FF0FF359E6804EB421351012F
:1049F000D3F80009002805DAD3F8000940F0804018
:104A0000C3F80009D3F8000B002805DAD3F8000B2F
:104A100040F08040C3F8000B013263189642C3F89F
:104A20000859C3F8085BE0D24FF00113C4F81C38F2
:104A300070BD000000EB8103D3F80CC02DE9F043FA
:104A4000DCF814204E1CD0F89050D2F800E005EBB2
:104A5000063605EB4118506870450AD30122D5F897
:104A6000343802FA01F123EA0101C5F83418BDE82F
:104A7000F083AEEB0003BCF81040A34228BF2346EE
:104A8000D8F81849A4B2B3EB840FF0D89468A4F115
:104A9000040959F8047F3760A4EB09071F44042F69
:104AA000F7D81C44034494605360D4E7890141F073
:104AB0002001016103699B06FCD41220FEF7EABFC6
:104AC00010B50A4C2046FEF7B5FA094BC4F89030F1
:104AD000084BC4F89430084C2046FEF7ABFA074B5D
:104AE000C4F89030064BC4F8943010BDF84700204D
:104AF00000000840D06500089448002000000440F1
:104B0000DC65000870B503780546012B5DD1494B83
:104B1000D0F89040984259D1474B0E216520D3F8E8
:104B2000D82042F00062C3F8D820D3F8002142F028
:104B30000062C3F80021D3F80021D3F8802042F0AE
:104B40000062C3F88020D3F8802022F00062C3F80E
:104B50008020D3F8803000F071FC384BE360384B94
:104B6000C4F800380023D5F89060C4F8003EC02394
:104B700023604FF40413A3633369002BFCDA012391
:104B80000C203361FEF786FF3369DB07FCD412206B
:104B9000FEF780FF3369002BFCDA00262846A6606A
:104BA000FFF71CFF6B68C4F81068DB68C4F8146872
:104BB000C4F81C68002B3AD1224BA3614FF0FF339D
:104BC0006361A36843F00103A36070BD1E4B98426C
:104BD000C8D1194B0E214D20D3F8D82042F00072D5
:104BE000C3F8D820D3F8002142F00072C3F80021A6
:104BF000D3F80021D3F8802042F00072C3F880205F
:104C0000D3F8802022F00072C3F88020D3F88020EF
:104C1000D3F8D82022F08062C3F8D820D3F800213E
:104C200022F08062C3F80021D3F8003193E7074BEC
:104C3000C3E700BFF847002000440258401400407A
:104C400003002002003C30C094480020083C30C0E3
:104C5000F8B5D0F89040054600214FF00066204698
:104C6000FFF724FFD5F8941000234FF001128F684E
:104C70004FF0FF30C4F83438C4F81C2804EB43125A
:104C800001339F42C2F80069C2F8006BC2F80809FC
:104C9000C2F8080BF2D20B68D5F89020C5F898300E
:104CA000636210231361166916F01006FBD11220FF
:104CB000FEF7F0FED4F8003823F4FE63C4F80038A1
:104CC000A36943F4402343F01003A3610923C4F80C
:104CD0001038C4F814380B4BEB604FF0C043C4F8E5
:104CE000103B094BC4F8003BC4F81069C4F8003904
:104CF000D5F8983003F1100243F48013C5F89820DA
:104D0000A362F8BDAC65000840800010D0F8902088
:104D100090F88A10D2F8003823F4FE6343EA0113B6
:104D2000C2F80038704700002DE9F84300EB81031A
:104D3000D0F890500C468046DA680FFA81F94801A5
:104D4000166806F00306731E022B05EB41134FF0A5
:104D5000000194BFB604384EC3F8101B4FF0010198
:104D600004F1100398BF06F1805601FA03F391692C
:104D700098BF06F5004600293AD0578A04F1580139
:104D8000374349016F50D5F81C180B430021C5F873
:104D90001C382B180127C3F81019A7405369611E4E
:104DA0009BB3138A928B9B08012A88BF5343D8F880
:104DB0009820981842EA034301F140022146C8F8BE
:104DC0009800284605EB82025360FFF76FFE08EB60
:104DD0008900C3681B8A43EA845348341E43640134
:104DE0002E51D5F81C381F43C5F81C78BDE8F88350
:104DF00005EB4917D7F8001B21F40041C7F8001B49
:104E0000D5F81C1821EA0303C0E704F13F030B4A5D
:104E10002846214605EB83035A60FFF747FE05EB62
:104E20004910D0F8003923F40043C0F80039D5F810
:104E30001C3823EA0707D7E70080001000040002AF
:104E4000D0F894201268C0F89820FFF7C7BD000082
:104E50005831D0F8903049015B5813F4004004D029
:104E600013F4001F0CBF0220012070474831D0F816
:104E7000903049015B5813F4004004D013F4001F34
:104E80000CBF02200120704700EB8101CB68196A3A
:104E90000B6813604B6853607047000000EB8103A0
:104EA00030B5DD68AA691368D36019B9402B84BF97
:104EB000402313606B8A1468D0F890201C4402EBE6
:104EC0004110013C09B2B4FBF3F46343033323F014
:104ED000030343EAC44343F0C043C0F8103B2B68CC
:104EE00003F00303012B0ED1D2F8083802EB411076
:104EF00013F4807FD0F8003B14BF43F0805343F09D
:104F00000053C0F8003B02EB4112D2F8003B43F0E3
:104F10000443C2F8003B30BD2DE9F041D0F8906069
:104F200005460C4606EB4113D3F8087B3A07C3F855
:104F3000087B08D5D6F814381B0704D500EB81038D
:104F4000DB685B689847FA071FD5D6F81438DB078B
:104F50001BD505EB8403D968CCB98B69488A5A689C
:104F6000B2FBF0F600FB16228AB91868DA689042A4
:104F70000DD2121AC3E90024202383F3118821469D
:104F80002846FFF78BFF84F31188BDE8F0810123E9
:104F900003FA04F26B8923EA02036B81CB68002BCE
:104FA000F3D021462846BDE8F041184700EB8103C5
:104FB0004A0170B5DD68D0F890306C692668E6600B
:104FC00056BB1A444FF40020C2F810092A6802F0B8
:104FD0000302012A0AB20ED1D3F8080803EB4214E7
:104FE00010F4807FD4F8000914BF40F0805040F0E6
:104FF0000050C4F8000903EB4212D2F8000940F057
:105000000440C2F800090122D3F8340802FA01F181
:105010000143C3F8341870BD19B9402E84BF402035
:10502000206020681A442E8A8419013CB4FBF6F4EF
:1050300040EAC44040F00050C6E700002DE9F041CE
:10504000D0F8906004460D4606EB4113D3F808797A
:10505000C3F80879FB071CD5D6F81038DA0718D53D
:1050600000EB8103D3F80CC0DCF81430D3F800E077
:10507000DA6896451BD2A2EB0E024FF000081A60C8
:10508000C3F80480202383F31188FFF78FFF88F390
:1050900011883B0618D50123D6F83428AB401342BB
:1050A00012D029462046BDE8F041FFF7C3BC0123DA
:1050B00003FA01F2038923EA02030381DCF80830D2
:1050C000002BE6D09847E4E7BDE8F0812DE9F84FE2
:1050D000D0F8905004466E69AB691E4016F48058B3
:1050E0006E6103D0BDE8F84FFEF714B8002E12DA57
:1050F000D5F8003E9F0705D0D5F8003E23F0030306
:10510000C5F8003ED5F80438204623F00103C5F861
:105110000438FEF72BF8300505D52046FFF75EFC76
:105120002046FEF713F8B1040CD5D5F8083813F073
:10513000060FEB6823F470530CBF43F4105343F491
:10514000A053EB60320704D56368DB680BB12046DF
:105150009847F30200F1BA80B70226D5D4F89090B0
:1051600000274FF0010A09EB4712D2F8003B03F485
:105170004023B3F5802F11D1D2F8003B002B0DDA7C
:1051800062890AFA07F322EA0303638104EB8703C7
:10519000DB68DB6813B13946204698470137D4F8FD
:1051A0009430FFB29B689F42DDD9F00619D5D4F840
:1051B0009000026AC2F30A1702F00F0302F4F01221
:1051C000B2F5802F00F0CC80B2F5402F09D104EB6E
:1051D0008303002200F58050DB681B6A974240F091
:1051E000B2803003D5F8185835D5E90303D500212E
:1051F0002046FFF791FEAA0303D501212046FFF7C1
:105200008BFE6B0303D502212046FFF785FE2F039B
:1052100003D503212046FFF77FFEE80203D50421D2
:105220002046FFF779FEA90203D505212046FFF7A6
:1052300073FE6A0203D506212046FFF76DFE2B029E
:1052400003D507212046FFF767FEEF0103D50821AC
:105250002046FFF761FE700340F1A980E90703D5FE
:1052600000212046FFF7EAFEAA0703D501212046C8
:10527000FFF7E4FE6B0703D502212046FFF7DEFEB1
:105280002F0703D503212046FFF7D8FEEE0603D5EE
:1052900004212046FFF7D2FEA80603D505212046AB
:1052A000FFF7CCFE690603D506212046FFF7C6FEB0
:1052B0002A0603D507212046FFF7C0FEEB0576D569
:1052C00020460821BDE8F84FFFF7B8BED4F890900B
:1052D00000274FF0010AD4F894305FFA87FB9B68EF
:1052E0009B453FF639AF09EB4B13D3F8002902F485
:1052F0004022B2F5802F24D1D3F80029002A20DAE9
:10530000D3F8002942F09042C3F80029D3F80029CD
:10531000002AFBDB5946D4F89000FFF7C7FB22892F
:105320000AFA0BF322EA0303238104EB8B03DB6805
:105330009B6813B159462046984759462046FFF7C7
:1053400079FB0137C7E7910701D1D0F80080072A20
:1053500002F101029CBF03F8018B4FEA18283DE7D8
:1053600004EB830300F58050DA68D2F818C0DCF84B
:105370000820DCE9001CA1EB0C0C00218F4208D1B5
:10538000DB689B699A683A449A605A683A445A6062
:1053900027E711F0030F01D1D0F800808C4501F10F
:1053A000010184BF02F8018B4FEA1828E6E7BDE847
:1053B000F88F000008B50348FFF788FEBDE80840F5
:1053C000FFF7AAB9F847002008B50348FFF77EFEAB
:1053D000BDE80840FFF7A0B994480020D0F890300D
:1053E00003EB4111D1F8003B43F40013C1F8003B3B
:1053F00070470000D0F8903003EB4111D1F800392C
:1054000043F40013C1F8003970470000D0F8903021
:1054100003EB4111D1F8003B23F40013C1F8003B2A
:1054200070470000D0F8903003EB4111D1F80039FB
:1054300023F40013C1F8003970470000090100F19E
:105440006043012203F56143C9B283F8001300F001
:105450001F039A4043099B0003F1604303F5614336
:10546000C3F880211A60704730B50433039C017281
:10547000002104FB0325C160C0E90653049B0363BC
:10548000059BC0E90000C0E90422C0E90842C0E968
:105490000A11436330BD00000022416AC260C0E9C6
:1054A0000411C0E90A226FF00101FEF77BBB000086
:1054B000D0E90432934201D1C2680AB9181D70477D
:1054C00000207047036919600021C2680132C26080
:1054D000C269134482699342036124BF436A036132
:1054E000FEF754BB38B504460D46E3683BB162692C
:1054F0000020131D1268A3621344E36207E0237ABD
:1055000033B929462046FEF731FB0028EDDA38BDD5
:105510006FF00100FBE70000C368C269013BC36094
:105520004369134482699342436124BF436A4361E0
:1055300000238362036B03B11847704770B52023C3
:10554000044683F31188866A3EB9FFF7CBFF054610
:1055500018B186F31188284670BDA36AE26A13F871
:10556000015B9342A36202D32046FFF7D5FF0023DD
:1055700083F31188EFE700002DE9F84F04460E464B
:10558000174698464FF0200989F311880025AA464E
:10559000D4F828B0BBF1000F09D141462046FFF7EF
:1055A000A1FF20B18BF311882846BDE8F88FD4E91C
:1055B0000A12A7EB050B521A934528BF9346BBF17D
:1055C000400F1BD9334601F1400251F8040B9142C0
:1055D00043F8040BF9D1A36A403640354033A36247
:1055E000D4E90A239A4202D32046FFF795FF8AF3B3
:1055F0001188BD42D8D289F31188C9E730465A468E
:10560000FBF742FFA36A5E445D445B44A362E7E7A5
:1056100010B5029C0433017204FB0321C460C0E98D
:1056200006130023C0E90A33039B0363049BC0E90C
:105630000000C0E90422C0E90842436310BD000035
:10564000026A6FF00101C260426AC0E904220022CE
:10565000C0E90A22FEF7A6BAD0E904239A4201D192
:10566000C26822B9184650F8043B0B60704700200E
:1056700070470000C3680021C2690133C3604369F9
:10568000134482699342436124BF436A4361FEF736
:105690007DBA000038B504460D46E3683BB1236986
:1056A00000201A1DA262E2691344E36207E0237A34
:1056B00033B929462046FEF759FA0028EDDA38BDFD
:1056C0006FF00100FBE7000003691960C268013A4E
:1056D000C260C269134482699342036124BF436A72
:1056E000036100238362036B03B118477047000016
:1056F00070B520230D460446114683F31188866A4F
:105700002EB9FFF7C7FF10B186F3118870BDA36AE9
:105710001D70A36AE26A01339342A36204D3E16974
:1057200020460439FFF7D0FF002080F31188EDE711
:105730002DE9F84F04460D46904699464FF0200A51
:105740008AF311880026B346A76A4FB94946204616
:10575000FFF7A0FF20B187F311883046BDE8F88F2E
:10576000D4E90A073A1AA8EB0607974228BF17465A
:10577000402F1BD905F1400355F8042B9D4240F8FA
:10578000042BF9D1A36A40364033A362D4E90A233B
:105790009A4204D3E16920460439FFF795FF8BF361
:1057A00011884645D9D28AF31188CDE729463A4671
:1057B000FBF76AFEA36A3D443E443B44A362E5E72F
:1057C000D0E904239A4217D1C3689BB1836A8BB195
:1057D000043B9B1A0ED01360C368013BC360C369CE
:1057E0001A4483699A42026124BF436A0361002319
:1057F00083620123184670470023FBE700F0F6B8E8
:10580000034B002258631A610222DA60704700BF1E
:10581000000C0040014B0022DA607047000C004091
:10582000014B5863704700BF000C0040014B586AA1
:10583000704700BF000C0040024B034A1A60034A45
:105840005A60704748490020D849002000000220D3
:10585000074B494210B55C68201A08401968821A43
:10586000914203D8944201D35A6010BD0020FCE756
:105870004849002008B5202383F31188FFF7E8FF8B
:10588000002383F3118808BD4B6843608B688360F5
:10589000CB68C3600B6943614B6903628B694362E8
:1058A0000B6803607047000008B5354B40F2FF708D
:1058B000D3F8E0100143C3F8E010D3F80821024305
:1058C0003048C3F80821304AD3F808311146FFF7B1
:1058D000DBFF00F5806002F11C01FFF7D5FF00F54A
:1058E000806002F13801FFF7CFFF00F5806002F120
:1058F0005401FFF7C9FF00F5806002F17001FFF766
:10590000C3FF00F5806002F18C01FFF7BDFF00F5D9
:10591000806002F1A801FFF7B7FF00F5806002F197
:10592000C401FFF7B1FF00F5806002F1E001FFF76D
:10593000ABFF00F5806002F1FC01FFF7A5FF02F567
:105940008C7100F58060FFF79FFF00F00BF90F4BA3
:10595000D3F8902242F00102C3F89022D3F89422A7
:1059600042F00102C3F894220522C3F898204FF0B8
:105970006052C3F89C20064AC3F8A02008BD00BFAF
:105980000044025800000258E865000800ED00E0FD
:105990001F00080308B500F0EFFAFEF72FF8104BD0
:1059A000D3F8DC2042F04002C3F8DC20D3F8042115
:1059B00022F04002C3F80421D3F80431094B1A68DD
:1059C00042F008021A601A6842F004021A60FEF7F8
:1059D00055FEFEF7BFFCBDE80840FEF75FBA00BF0A
:1059E000004402580018024870470000114BD3F8D9
:1059F000E82042F00802C3F8E820D3F8102142F072
:105A00000802C3F810210C4AD3F81031D36B43F0CD
:105A10000803D363C722094B9A624FF0FF32DA6260
:105A200000229A615A63DA605A6001225A611A6050
:105A3000704700BF004402580010005C000C00409A
:105A4000094A08B51169D3680B40D9B29B076FEAC0
:105A50000101116107D5202383F31188FDF7FEFFB3
:105A6000002383F3118808BD000C004008B53C4BAF
:105A70004FF0FF31D3F8802062F00042C3F880205D
:105A8000D3F8802002F00042C3F88020D3F88020B1
:105A9000D3F88420C3F88410D3F884200022C3F8FC
:105AA0008420D3F88400D86F40F0FF4040F4FF001A
:105AB00040F43F5040F03F00D867D86F20F0FF40DF
:105AC00020F4FF0020F43F5020F03F00D867D86F4B
:105AD000D3F888006FEA40506FEA5050C3F888004E
:105AE000D3F88800C0F30A00C3F88800D3F8880010
:105AF000D3F89000C3F89010D3F89000C3F890202A
:105B0000D3F89000D3F89400C3F89410D3F894001D
:105B1000C3F89420D3F89400D3F89800C3F89810F1
:105B2000D3F89800C3F89820D3F89800D3F88C00E5
:105B3000C3F88C10D3F88C00C3F88C20D3F88C00F9
:105B4000D3F89C00C3F89C10D3F89C10C3F89C2099
:105B5000D3F89C30FEF7E8FEBDE8084000F0DCB961
:105B600000440258614B0122C3F80821604BD3F86E
:105B7000F42042F00202C3F8F420D3F81C2142F0D2
:105B80000202C3F81C210222D3F81C31594BDA60FF
:105B90005A689104FCD5584A1A6001229A60574A03
:105BA000DA6000221A614FF440429A61514B9A69BF
:105BB0009204FCD51A6842F480721A604C4B1A6F3A
:105BC00012F4407F04D04FF480321A6700221A6723
:105BD0001A6842F001021A60454B1A685007FCD55A
:105BE00000221A611A6912F03802FBD101211960F2
:105BF0004FF0804159605A67414ADA62414A1A615E
:105C00001A6842F480321A60394B1A689103FCD545
:105C10001A6842F480521A601A689204FCD53A4A13
:105C20003A499A6200225A6319633949DA639963DF
:105C30005A64384A1A64384ADA621A6842F0A8523A
:105C40001A602B4B1A6802F02852B2F1285FF9D182
:105C500048229A614FF48862DA6140221A622F4A20
:105C6000DA644FF080521A652D4A5A652D4A9A65BA
:105C700032232D4A1360136803F00F03022BFAD16D
:105C80001B4B1A6942F003021A611A6902F03802CA
:105C9000182AFAD1D3F8DC2042F00052C3F8DC20F5
:105CA000D3F8042142F00052C3F80421D3F80421B0
:105CB000D3F8DC2042F08042C3F8DC20D3F8042182
:105CC00042F08042C3F80421D3F80421D3F8DC2049
:105CD00042F00042C3F8DC20D3F8042142F0004235
:105CE000C3F80421D3F80431704700BF008000518D
:105CF000004402580048025800C000F002000001B1
:105D00000000FF01008890081210200063020901C2
:105D10002C02040047040508FD0BFF0120000020B1
:105D20000010E00000010100002000524FF0B042DE
:105D300008B5D2F8883003F00103C2F8883023B1E7
:105D4000044A13680BB150689847BDE80840FEF755
:105D5000E3BC00BF504900204FF0B04208B5D2F874
:105D6000883003F00203C2F8883023B1044A9368F4
:105D70000BB1D0689847BDE80840FEF7CDBC00BF26
:105D8000504900204FF0B04208B5D2F8883003F0F7
:105D90000403C2F8883023B1044A13690BB1506977
:105DA0009847BDE80840FEF7B7BC00BF5049002047
:105DB0004FF0B04208B5D2F8883003F00803C2F8BB
:105DC000883023B1044A93690BB1D0699847BDE884
:105DD0000840FEF7A1BC00BF504900204FF0B04280
:105DE00008B5D2F8883003F01003C2F8883023B128
:105DF000044A136A0BB1506A9847BDE80840FEF7A1
:105E00008BBC00BF504900204FF0B04310B5D3F811
:105E1000884004F47872C3F88820A30604D5124A97
:105E2000936A0BB1D06A9847600604D50E4A136B8B
:105E30000BB1506B9847210604D50B4A936B0BB1FD
:105E4000D06B9847E20504D5074A136C0BB1506C30
:105E50009847A30504D5044A936C0BB1D06C9847BE
:105E6000BDE81040FEF758BC504900204FF0B04349
:105E700010B5D3F8884004F47C42C3F8882062054A
:105E800004D5164A136D0BB1506D9847230504D500
:105E9000124A936D0BB1D06D9847E00404D50F4AB8
:105EA000136E0BB1506E9847A10404D50B4A936E44
:105EB0000BB1D06E9847620404D5084A136F0BB13A
:105EC000506F9847230404D5044A936F0BB1D06FE9
:105ED0009847BDE81040FEF71FBC00BF50490020A6
:105EE00008B50348FCF708FCBDE80840FEF714BC01
:105EF000E424002008B50348FCF7AEFCBDE80840E8
:105F0000FEF70ABC0425002008B5FFF799FDBDE89F
:105F10000840FEF701BC0000062108B50846FFF75F
:105F20008DFA06210720FFF789FA06210820FFF7DE
:105F300085FA06210920FFF781FA06210A20FFF7DA
:105F40007DFA06211720FFF779FA06212820FFF7AE
:105F500075FA09217A20FFF771FA0A215C20FFF710
:105F60006DFA07213220FFF769FA0C212520BDE8E0
:105F70000840FFF763BA000008B5FFF777FD00F0AF
:105F80000FF8FCF77BFEFDF753F8FCF725FFFDF754
:105F9000E5FAFFF729FDBDE80840FFF72FBC000038
:105FA0000023054A19460133102BC2E9001102F102
:105FB0000802F8D1704700BF504900200B46014647
:105FC000184600F027B80000FEF7FCB9FFF7FCBF49
:105FD000012838BF012010B504462046FEF7B2F96B
:105FE00030B900F007F808B900F00CF88047F4E782
:105FF00010BD0000024B1868BFF35B8F704700BFF5
:10600000D049002008B5062000F04AF80120FDF72D
:1060100093FE000010B5054C13462CB10A4601460C
:106020000220AFF3008010BD2046FCE70000000016
:1060300010B501390244904201D1002005E00378F7
:1060400011F8014FA34201D0181B10BD0130F2E737
:106050001F2938B504460D4604D9162303604FF0B6
:10606000FF3038BD426C12B152F821304BB9204696
:1060700000F030F82A4601462046BDE8384000F0DE
:1060800017B8012B0AD0591C03D116230360012035
:10609000E7E7002442F82540284698470020E0E73B
:1060A000024B01461868FFF7D3BF00BF64220020EF
:1060B00038B5074D00230446084611462B60FDF70E
:1060C0003FFE431C02D12B6803B1236038BD00BFE3
:1060D000D4490020FDF72EBE034611F8012B03F82A
:1060E000012B002AF9D170470000000001000000D8
:1060F000000100010000000000000000000000009E
:1061000052657175657374656420746F2065726182
:106110007365206D6F7265207468616E20776520ED
:1061200063616E0A00457261736520436F6D6D6136
:106130006E642052656365697665640A0050435455
:1061400020444F4E453A2025640A000053544D33F5
:106150003248373F3F3F0053544D33324837343392
:106160002F3735330000000001105A00031059008A
:106170000120580003205600773235712D64747267
:10618000000000000000000000000000000000000F
:1061900000000000F9160008251A0008251A00085A
:1061A000FD16000801170008051700080917000868
:1061B000251A0008251A0008251A000821170008CA
:1061C000251700083D17000845170008511700085B
:1061D0005517000859170008E424002001000000AA
:1061E0000000000000000000791800089118000865
:1061F000F916000865170008C5180008811700087F
:106200005D1900088D190008091700087D1700089E
:1062100069170008791700082117000825170008DA
:106220003D170008451700085117000855170008CA
:10623000591700080000000000000000F9170008CE
:106240005D17000861170008534644500000000025
:106250004A454445433A204661696C656420746F41
:106260002064657465637420666C6173682064657E
:10627000766963653A2025730A004A454445433AE6
:10628000204661696C656420746F20636F6E666977
:106290006720666C617368206465766963653A207F
:1062A00025730A004A454445433A204465746563B2
:1062B00074656420466C6173682044657669636523
:1062C0003A2025730A0045787420466C6173682073
:1062D0004E6F7420466F756E642100006D74323508
:1062E0007100773235710000DC62000820BA0000CE
:1062F000E2620008EF40000078610008EF700000E3
:1063000000000000000000000521000865230008CF
:10631000411A0008451A0008ED1A0008CD220008AD
:10632000491A00084D1A0008C5210008BD1A0008C6
:1063300025220008291F0008551A0008511A0008D4
:10634000F5230008B51A0008000000000000000056
:10635000B9240008C1240008A5240008AD240008C1
:10636000D1240008D52400084D444D4120666169C0
:106370006C757265000000000096000000000000CF
:10638000000000000000000000000000000000000D
:1063900000000000452C0008312C00086D2C00087E
:1063A000592C0008652C0008512C00083D2C0008D1
:1063B000292C0008792C000800000000552D000849
:1063C000412D00087D2D0008692D0008752D00085D
:1063D000612D00084D2D0008392D0008892D000879
:1063E0000000000001000000000000006D61696E07
:1063F0000000000069646C6500000000F4630008A0
:10640000C8290020402B002001000000F9390008B5
:10641000000000004172647550696C6F7400254281
:106420004F415244252D424C002553455249414C81
:10643000250000000200000000000000752F000889
:10644000E52F000840004000E8430020F84300200A
:106450000200000000000000030000000000000037
:106460002D3000080000000010000000084400204B
:10647000000000000100000000000000F8470020BC
:1064800001010200393E0008493D0008E53D0008D1
:10649000C93D0008430000009C6400080902430055
:1064A000020100C0320904000001020201000524BB
:1064B0000010010524010001042402020524060045
:1064C00001070582030800FF09040100020A000019
:1064D000000705010240000007058102400000009E
:1064E00012000000E86400081201100102000040E0
:1064F00009124157000201020301000004030904CC
:1065000025424F41524425005350526163696E67E2
:106510004837003031323334353637383941424329
:106520004445460000000020000002000200000078
:106530000000003000000400000000000000002403
:1065400000000800040000000004000000FC00003F
:106550000200000000000430008000000000000085
:10656000000000380000010001000000400000525F
:1065700080000052C0000052000100524001005251
:1065800080010052C001005200020052400200523D
:1065900080020052C0020052000300524003005229
:1065A00080030052C00300520004005200000000AB
:1065B0008131000839340008E5340008400040000B
:1065C00030490020304900200100000040490020EF
:1065D00080000000400100000800000000010000F1
:1065E00000040000080000000000806A00000000B5
:1065F000AAAAAAAA00000064FFFF00000000000091
:1066000000A00A00240020A100000000AAAAAAAA53
:1066100000000051FFFF00000009000000090044D5
:106620000000000000000000AAAAAAAA00000000C2
:10663000FFFF000000000000000000000000800AD2
:1066400000000000AAAAAAAA00000000FFFF0000A4
:106650000000000000909900600040000000000071
:10666000AAAAAAAA00004000F7FF00000009000043
:10667000000000000000000000000000AAAAAAAA72
:1066800000000000FFFF000000000000000000000C
:106690000000000000000000AAAAAAAA0000000052
:1066A000FFFF0000000000000000000000000000EC
:1066B00000000000AAAAAAAA00000000FFFF000034
:1066C00000000000000000000000000000000000CA
:1066D000AAAAAAAA00000000FFFF00000000000014
:1066E000000000000000000000000000AAAAAAAA02
:1066F00000000000FFFF000000000000000000009C
:106700000000000000000000AAAAAAAA00000000E1
:10671000FFFF00000000000000000000C49BFF7F9E
:106720000100000000000000240400000000000040
:10673000000000000000E900FF000000402B0020E6
:1067400004250020000000004C6100083F0000000C
:1067500050040000576100083F0000000096000050
:10676000000008009600000000080000040000007F
:10677000FC640008000000000000000000000000B1
:10678000000000000000000000000000682200205F
:1067900000000000000000000000000000000000F9
:1067A00000000000000000000000000000000000E9
:1067B00000000000000000000000000000000000D9
:1067C00000000000000000000000000000000000C9
:1067D00000000000000000000000000000000000B9
:1067E00000000000000000000000000000000000A9
:00000001FF
